:0200000480007A
:100000006F00C004732F2034930F8000630AFF0336
:10001000930F90006306FF03930FB0006302FF038A
:10002000170F0080130F0FFE63040F0067000F000F
:10003000732F203463540F006F004000136E9E53E3
:10004000171F00002320CFFD6FF09FFF732540F1A5
:100050006310050073251030635805000F00F00F82
:10006000130E100073000000130E00009702000032
:10007000938282F973905230735020307350303035
:1000800073504030970200809382C2F7638C020065
:10009000739052109302B01A739022307323203061
:1000A000E39E62F873500030970200009382420191
:1000B00073901234732540F17300203093000000D8
:1000C00013010000B3812040930E0000130E2000A6
:1000D0006396D14B9300100013011000B3812040B0
:1000E000930E0000130E3000639AD1499300300044
:1000F00013017000B3812040930EC0FF130E400027
:10010000639ED147930000003781FFFFB3812040F9
:10011000B78E0000130E50006392D147B7000080E5
:1001200013010000B3812040B70E0080130E600061
:100130006396D145B70000803781FFFFB38120402F
:10014000B78E0080130E7000639AD14393000000B5
:10015000378100001301F1FFB3812040B78EFFFF0C
:10016000938E1E00130E8000639AD141B700008069
:100170009380F0FF13010000B3812040B70E008090
:10018000938EFEFF130E9000639AD13FB70000805C
:100190009380F0FF378100001301F1FFB38120400D
:1001A000B78EFF7F130EA000639AD13DB700008089
:1001B000378100001301F1FFB3812040B78EFF7F2C
:1001C000938E1E00130EB000639AD13BB7000080DF
:1001D0009380F0FF3781FFFFB3812040B78E00800E
:1001E000938EFEFF130EC000639AD1399300000076
:1001F0001301F0FFB3812040930E1000130ED000C6
:10020000639ED1379300F0FF13011000B3812040AB
:10021000930EE0FF130EE0006392D1379300F0FFDE
:100220001301F0FFB3812040930E0000130EF00085
:100230006396D1359300D0001301B000B380204005
:10024000930E2000130E0001639AD0339300E00058
:100250001301B00033812040930E3000130E1001C3
:10026000631ED1319300D000B3801040930E000084
:10027000130E20016394D031130200009300D000CC
:100280001301B000B3812040138301001302120058
:1002900093022000E31452FE930E2000130E30014F
:1002A000631ED32D130200009300E0001301B00081
:1002B000B3812040130000001383010013021200D9
:1002C00093022000E31252FE930E3000130E400101
:1002D0006316D32B130200009300F0001301B0004B
:1002E000B3812040130000001300000013830100BD
:1002F0001302120093022000E31052FE930E4000FE
:10030000130E5001631CD327130200009300D0008A
:100310001301B000B38120401302120093022000A9
:10032000E31652FE930E2000130E60016398D12550
:10033000130200009300E0001301B000130000005E
:10034000B38120401302120093022000E31452FEF6
:10035000930E3000130E70016392D123130200003C
:100360009300F0001301B000130000001300000020
:10037000B38120401302120093022000E31252FEC8
:10038000930E4000130E8001639AD11F13020000E8
:100390009300D000130000001301B000B38120408F
:1003A0001302120093022000E31452FE930E200069
:1003B000130E90016394D11D130200009300E0001E
:1003C000130000001301B00013000000B3812040AF
:1003D0001302120093022000E31252FE930E30002B
:1003E000130EA001639CD119130200009300F000CA
:1003F00013000000130000001301B000B38120407F
:100400001302120093022000E31252FE930E4000EA
:10041000130EB0016394D117130200001301B00052
:100420009300D000B38120401302120093022000F9
:10043000E31652FE930E2000130EC0016390D115F7
:10044000130200001301B0009300E000130000004D
:10045000B38120401302120093022000E31452FEE5
:10046000930E3000130ED001639AD11113020000D5
:100470001301B0009300F00013000000130000000F
:10048000B38120401302120093022000E31252FEB7
:10049000930E4000130EE0016392D10F130200008F
:1004A0001301B000130000009300D000B38120407E
:1004B0001302120093022000E31452FE930E200058
:1004C000130EF001639CD10B130200001301B00066
:1004D000130000009300E00013000000B3812040EF
:1004E0001302120093022000E31252FE930E30001A
:1004F000130E00026394D109130200001301B0002F
:1005000013000000130000009300F000B3812040AE
:100510001302120093022000E31252FE930E4000D9
:10052000130E1002639CD105930010FF330110409D
:10053000930EF000130E20026312D1059300000207
:1005400033810040930E0002130E30026318D10372
:10055000B3000040930E0000130E40026390D003DE
:10056000930000011301E00133802040930E00004E
:10057000130E50026314D001631CC0010F00F00F72
:1005800063000E00131E1E00136E1E007300000099
:100590000F00F00F130E100073000000731000C066
:1005A000000000000000000000000000000000004B
:1005B000000000000000000000000000000000003B
:0405C0000000000037
:1010000000000000000000000000000000000000E0
:1010100000000000000000000000000000000000D0
:1010200000000000000000000000000000000000C0
:1010300000000000000000000000000000000000B0
:081040000000000000000000A8
:040000058000200057
:00000001FF
